:100000000C945B000C947F030C94AC030C94830061
:100010000C9483000C9483000C9483000C94830054
:100020000C9483000C9483000C9483000C94830044
:100030000C9483000C9483000C9483000C94830034
:100040000C94D9030C9483000C9495050C948300B4
:100050000C9483000C9483000C9483000C94830014
:100060000C9483000C948300000024272A000025B0
:10007000282B000023262904040404040404040299
:100080000202020202030303030303010204081035
:100090002040800102040810200102040810200002
:1000A0000000070002010000030406000000000039
:1000B00000000000950211241FBECFEFD4E0DEBF88
:1000C000CDBF11E0A0E0B1E0ECE7FCE002C005909C
:1000D0000D92A231B107D9F712E0A2E1B1E001C05F
:1000E0001D92AA3FB107E1F710E0C6EBD0E004C0D3
:1000F0002297FE010E943806C43BD107C9F70E942F
:100100008E020C943C060C94000040E051EE60E03E
:1001100070E084E692E00E94A60264E670E080E06F
:1001200090E00E94490461E0809100010E94BB04BC
:100130000895BF92CF92DF92EF92FF920F931F9399
:10014000DF93CF93CDB7DEB72A970FB6F894DEBF13
:100150000FBECDBF6B01DE011196E2E0F1E02AE0B7
:1001600001900D922150E1F79C0189589F4FFC01AD
:10017000849125573F4FF901B490E82FF0E0EE0F3E
:10018000FF1FEC0FFD1F0181128190E2E92EF12C7F
:10019000E00EF11EF80180A18B2980A38AE090E097
:1001A0000E947304F894F80180A19B2D90958923F7
:1001B00080A300000000000000000000000000001C
:1001C000000000000000000000000000000000002F
:1001D000000000000000000000000000000000001F
:1001E000000000000000000000000000000000000F
:1001F00000000000000000000000000000000000FF
:1002000000000000000000000000000000000000EE
:10021000000020E030E0C0FE04C0F70180818B299F
:1002200003C0F70180818923808300000000000063
:1002300000000000000000000000000000000000BE
:1002400000000000000000000000000000000000AE
:10025000000000000000000000000000000000009E
:10026000000000000000000000000000000000008E
:10027000000000000000000000000000000000007E
:10028000000000000000000000002F5F3F4F2830FA
:10029000310519F0D594C794BECFF80180A18B2900
:1002A00080A378942A960FB6F894DEBF0FBECDBF18
:1002B000CF91DF911F910F91FF90EF90DF90CF9042
:1002C000BF900895CF93DF9360E0809100010E947A
:1002D000D90484E690E00E94730410922402C0E0E6
:1002E000D0E08091000190910101C034D10531F03E
:1002F000FE01EC5DFD4F608170E002C060E070E0E7
:100300000E9499002196C134D10559F7DF91CF9110
:10031000089584E692E00E94A302882309F4ADC008
:1003200084E692E00E94A002AC01909313018093B6
:100330001201893D910549F48091140190911501B4
:10034000892B19F481E090E00BC0209114013091C9
:1003500015012130310549F44093190182E090E004
:1003600090931501809314010EC0C9010297049760
:1003700050F4F901E65EFE4F40832F5F3F4F30930C
:100380001501209314018091140190911501069795
:1003900009F073C0109215011092140120911C01F4
:1003A00030911D0150911E01832F820F850F809384
:1003B000180190911F01409119019817F1F44423FD
:1003C00039F420932401309325015093260155C020
:1003D000842F90E0FC01EE0FFF1FE80FF91FEC5D8A
:1003E000FE4F218332830196FC01EE0FFF1FE80FC1
:1003F000F91FEC5DFE4F508340C050E060E070E0BC
:1004000020E030E084E692E00E946A0340911C0103
:1004100050E060E070E020E030E084E692E00E948E
:100420006A0340911D0150E060E070E020E030E0A0
:1004300084E692E00E946A0340911E0150E060E071
:1004400070E020E030E084E692E00E946A03409190
:100450001F0150E060E070E020E030E084E692E0D0
:100460000E946A034091180150E060E070E020E0D3
:1004700030E084E692E00E946A038091140190913A
:100480001501892B09F049C0809119018823D9F4FD
:100490001092170110921601A4E2B1E080E090E002
:1004A0000AC02C91E82F803420F4F0E0EC5DFD4F81
:1004B000208301961196833091059CF39093170148
:1004C0008093160128C090E09C01220F331F280F53
:1004D000391F2F5F3F4F309317012093160101966C
:1004E000AC01440F551F480F591FD901AC5DBE4FD9
:1004F0000BC08C91E22F203420F4F0E0EC5DFD4F36
:1005000080832F5F3F4F11964217530794F7309324
:100510001701209316010E94620108950E94810430
:100520000E9485000E948901FDCF80E191E09093B7
:100530006502809364020895862F0E945D050895E8
:100540000E94760508950E9465050895CB01BA01C1
:100550000E94240508952F923F924F925F926F92CE
:100560007F928F929F92AF92BF92CF92DF92EF9243
:10057000FF920F931F93DF93CF93CDB7DEB7A09772
:100580000FB6F894DEBF0FBECDBF1C016A017B0120
:10059000411551056105710549F4DC01ED91FC91AE
:1005A0000190F081E02D60E3099554C088249924DE
:1005B0005401422E55246624772401E010E00C0FEC
:1005C0001D1F080D191DC701B601A30192010E944C
:1005D000E505F80160830894811C911CA11CB11CE5
:1005E000C701B601A30192010E94E505C901DA0124
:1005F0006C017D01C114D104E104F104F1F681E044
:10060000E82EF12CEC0EFD1EE80CF91C3E010894BE
:10061000611C711CD501C4010197A109B1096C01CC
:10062000C818D90814C0F601EE0DFF1D60816A30AC
:1006300010F4605D01C0695CD101ED91FC91019005
:10064000F081E02DC10109950894E108F1086E14CC
:100650007F0449F7A0960FB6F894DEBF0FBECDBF5A
:10066000CF91DF911F910F91FF90EF90DF90CF908E
:10067000BF90AF909F908F907F906F905F904F90C2
:100680003F902F900895EF92FF920F931F93CF9377
:10069000DF93EC017A018B0177FF0FC0E881F981CC
:1006A0000190F081E02D6DE2099510950095F09490
:1006B000E094E11CF11C011D111D2AE0B801A70105
:1006C000CE010E94AB02DF91CF911F910F91FF905D
:1006D000EF900895DC012115310541F4ED91FC9175
:1006E0000190F081E02D642F099508952A3031059D
:1006F00019F40E94430308950E94AB0208951F92CB
:100700000F920FB60F9211242F933F934F935F9345
:100710006F937F938F939F93AF93BF93EF93FF93C9
:100720008091660290916702892B29F0E091660220
:10073000F09167020995FF91EF91BF91AF919F9161
:100740008F917F916F915F914F913F912F910F907A
:100750000FBE0F901F9018951F920F920FB60F9219
:1007600011242F933F934F935F936F937F938F93B6
:100770009F93AF93BF93EF93FF9380916802909103
:100780006902892B29F0E0916802F09169020995CC
:10079000FF91EF91BF91AF919F918F917F916F9159
:1007A0005F914F913F912F910F900FBE0F901F902F
:1007B00018951F920F920FB60F9211242F938F93BB
:1007C0009F93AF93BF9380916A0290916B02A09127
:1007D0006C02B0916D020196A11DB11D80936A0259
:1007E00090936B02A0936C02B0936D0280916E02A5
:1007F00090916F02A0917002B09171028050904C64
:10080000AF4FBF4F80936E0290936F02A093700220
:10081000B093710227C080916E0290916F02A091F7
:100820007002B091710280589E43A040B040809306
:100830006E0290936F02A0937002B0937102809148
:10084000720290917302A0917402B09175020196A8
:10085000A11DB11D8093720290937302A093740244
:10086000B093750280916E0290916F02A091700218
:10087000B091710281589E43A040B04060F6BF9194
:10088000AF919F918F912F910F900FBE0F901F905E
:100890001895EF92FF920F931F937B018C018FB7F6
:1008A000F8944091720250917302609174027091B9
:1008B00075028FBF2FB7F8948091720290917302E6
:1008C000A0917402B09175022FBF841B950BA60BEB
:1008D000B70BE816F9060A071B0760F71F910F917F
:1008E000FF90EF900895019759F0FC01EE0FFF1F64
:1008F000EE0FFF1F32978FB7F8943197F1F78FBF44
:100900000895789484B5826084BD84B5816084BD87
:1009100085B5826085BD85B5816085BDEEE6F0E078
:10092000808181608083E1E8F0E080818260808363
:10093000808181608083E0E8F0E080818160808355
:10094000E1EBF0E0808184608083E0EBF0E0808187
:1009500081608083EAE7F0E0808184608083808129
:1009600082608083808181608083808180688083D1
:100970001092C1000895282F30E0C90185579F4F7C
:10098000FC01949129583F4FF9018491882381F00B
:10099000E82FF0E0E859FF4FE491F0E0662329F4F6
:1009A000808190958923808308958081892B80831D
:1009B0000895482F50E0CA0181569F4FFC012491B1
:1009C000CA0185579F4FFC01949149585F4FFA0126
:1009D00034913323C1F1222331F1233021F480916A
:1009E00080008F7705C0243031F4809180008F7DA6
:1009F0008093800018C0213019F484B58F7704C02B
:100A0000223021F484B58F7D84BD0DC0263021F4C1
:100A10008091B0008F7705C0273029F48091B00015
:100A20008F7D8093B000E32FF0E0E359FF4FE49116
:100A3000F0E0662329F480819095892380830895CE
:100A40008081892B80830895EF92FF920F931F93EB
:100A50007B018C0122E030E040E050E00E9407067C
:100A6000205C3D4B404F5F4FCA01B901A80197017F
:100A70000E940706C901DA010197A109B109292FCE
:100A80003A2F4B2F552747FD5A950196A11DB11DB1
:100A90002093C50081508093C400E1ECF0E0808198
:100AA000806180838081886080838081806880838A
:100AB0001F910F91FF90EF900895982F8091C000A3
:100AC00085FFFCCF9093C6000895809176029091A7
:100AD000770280589F4F2091780230917902821BD3
:100AE000930B60E870E00E94D2050895409178026F
:100AF0005091790280917602909177028417950740
:100B000019F42FEF3FEF0FC0FA01E658FD4F208197
:100B1000CA01019660E870E00E94D20590937902C4
:100B20008093780230E0C90108951F920F920FB6AA
:100B30000F9211242F933F934F935F936F937F9363
:100B40008F939F93AF93BF93EF93FF934091C60012
:100B5000E0917602F0917702CF01019660E870E0B3
:100B60000E94D2059C018091780290917902281709
:100B7000390739F0E658FD4F4083309377022093D0
:100B80007602FF91EF91BF91AF919F918F917F91ED
:100B90006F915F914F913F912F910F900FBE0F90EA
:100BA0001F90189597FB092E07260AD077FD04D0D1
:100BB00049D006D000201AF4709561957F4F0895B2
:100BC000F6F7909581959F4F0895A1E21A2EAA1BE2
:100BD000BB1BFD010DC0AA1FBB1FEE1FFF1FA217ED
:100BE000B307E407F50720F0A21BB30BE40BF50BEA
:100BF000661F771F881F991F1A9469F76095709573
:100C0000809590959B01AC01BD01CF01089597FBA4
:100C1000092E05260ED057FD04D0D7DF0AD0001CC0
:100C200038F450954095309521953F4F4F4F5F4F89
:100C30000895F6F790958095709561957F4F8F4F49
:100C40009F4F0895AA1BBB1B51E107C0AA1FBB1FE2
:100C5000A617B70710F0A61BB70B881F991F5A9548
:100C6000A9F780959095BC01CD010895EE0FFF1F67
:0C0C70000590F491E02D0994F894FFCF5A
:100C7C00080000000000050008000B000000000048
:020C8C009C02C8
:00000001FF
